******************************************************************************
                  TI ARM Linker PC v5.2.5                      
******************************************************************************
>> Linked Wed Dec 14 09:39:53 2016

OUTPUT FILE NAME:   <FEE_E2E_3137ZWT.out>
ENTRY POINT SYMBOL: "_c_int00"  address: 0000d024


MEMORY CONFIGURATION

         name            origin    length      used     unused   attr    fill
----------------------  --------  ---------  --------  --------  ----  --------
  VECTORS               00000000   00000020  00000020  00000000     X
  FLASH0                00000020   0017ffe0  00011584  0016ea5c  R  X
  FLASH1                00180000   00180000  00000000  00180000  R  X
  STACKS                08000000   00001500  00000000  00001500  RW  
  RAM                   08001500   0003eb00  00000215  0003e8eb  RW  


SEGMENT ALLOCATION MAP

run origin  load origin   length   init length attrs members
----------  ----------- ---------- ----------- ----- -------
00000000    00000000    000115a8   000115a8    r-x
  00000000    00000000    00000020   00000020    r-x .intvecs
  00000020    00000020    0000e418   0000e418    r-x .text
  0000e438    0000e438    00002ec0   00002ec0    r-x FEE_TEXT_SECTION
  000112f8    000112f8    00000180   00000180    r-- .const
  00011478    00011478    000000dc   000000dc    r-- FEE_CONST_SECTION
  00011558    00011558    00000050   00000050    r-- .cinit
08001500    08001500    00000218   00000000    rw-
  08001500    08001500    00000131   00000000    rw- FEE_DATA_SECTION
  08001634    08001634    0000007e   00000000    rw- .data
  080016b2    080016b2    00000066   00000000    rw- .bss


SECTION ALLOCATION MAP

 output                                  attributes/
section   page    origin      length       input sections
--------  ----  ----------  ----------   ----------------
.intvecs   0    00000000    00000020     
                  00000000    00000020     sys_intvecs.obj (.intvecs)

.text      0    00000020    0000e418     
                  00000020    000057f0     ti_fee_util.obj (.text)
                  00005810    00002cdc     sys_selftest.obj (.text)
                  000084ec    00001750     ti_fee_ini.obj (.text)
                  00009c3c    000010c4     ti_fee_main.obj (.text)
                  0000ad00    00000b28     system.obj (.text)
                  0000b828    00000898     sys_vim.obj (.text)
                  0000c0c0    00000630     pinmux.obj (.text)
                  0000c6f0    000005e8     esm.obj (.text)
                  0000ccd8    0000034c     sys_core.obj (.text)
                  0000d024    00000298     sys_startup.obj (.text:retain)
                  0000d2bc    00000294     sys_vim.obj (.text:retain)
                  0000d550    00000260     F021_API_CortexR4_BE.lib : FlashStateMachine.InitializeFlashBanks.obj (.text:Fapi_initializeFlashBanks)
                  0000d7b0    0000017c                              : FlashStateMachine.SetActiveBank.obj (.text:Fapi_setActiveFlashBank)
                  0000d92c    00000154     sys_main.obj (.text)
                  0000da80    00000114     esm.obj (.text:retain)
                  0000db94    000000e8     dabort.obj (.text)
                  0000dc7c    000000e0     sys_pmu.obj (.text)
                  0000dd5c    0000009c     rtsv7R4_T_be_v3D16_eabi.lib : memcpy_t2.obj (.text)
                  0000ddf8    00000094     F021_API_CortexR4_BE.lib : BlankCheck.obj (.text:Fapi_doBlankCheck)
                  0000de8c    00000080                              : FlashStateMachine.EnableEepromSectors.obj (.text:Fapi_enableEepromBankSectors)
                  0000df0c    0000007a     rtsv7R4_T_be_v3D16_eabi.lib : memset_t2.obj (.text)
                  0000df86    00000002     --HOLE-- [fill = 0]
                  0000df88    0000006c     notification.obj (.text)
                  0000dff4    0000006c     rtsv7R4_T_be_v3D16_eabi.lib : autoinit.obj (.text)
                  0000e060    0000006a                                 : copy_decompress_rle.obj (.text)
                  0000e0ca    0000005e     F021_API_CortexR4_BE.lib : Read.LoopDword.obj (.text:_Fapi_loopRegionForValue)
                  0000e128    00000050                              : FlashStateMachine.Hercules.IsEccAddress.obj (.text:Fapi_isAddressEcc)
                  0000e178    0000004c     rtsv7R4_T_be_v3D16_eabi.lib : cpy_tbl.obj (.text)
                  0000e1c4    00000044     F021_API_CortexR4_BE.lib : FlashStateMachine.EnableEepromSectors.obj (.text:_Fapi_EnableSectors)
                  0000e208    00000040     rtsv7R4_T_be_v3D16_eabi.lib : exit.obj (.text)
                  0000e248    0000003c     F021_API_CortexR4_BE.lib : FlashStateMachine.IssueFsmCommand.obj (.text:_Fapi_issueFsmCommand)
                  0000e284    00000036                              : Utilities.CalculateFletcher.obj (.text:Fapi_calculateFletcherChecksum)
                  0000e2ba    00000002     --HOLE-- [fill = 0]
                  0000e2bc    00000030                              : Async.WithAddress.obj (.text:Fapi_issueAsyncCommandWithAddress)
                  0000e2ec    00000030                              : Utilities.WaitDelay.obj (.text:Fapi_waitDelay)
                  0000e31c    0000002c                              : Read.Common.obj (.text:_Fapi_readDword)
                  0000e348    0000002a                              : Async.obj (.text:Fapi_issueAsyncCommand)
                  0000e372    00000022                              : Read.FlushPipeline.obj (.text:Fapi_flushPipeline)
                  0000e394    0000001c                              : FlashStateMachine.InitializeFlashBanks.obj (.text:_Fapi_divideUnsignedLong)
                  0000e3b0    00000014     rtsv7R4_T_be_v3D16_eabi.lib : _lock.obj (.text)
                  0000e3c4    00000010     F021_API_CortexR4_BE.lib : Utilities.GetNumberOfSectors.obj (.text:Fapi_getNumberOfBankSectors)
                  0000e3d4    00000010                              : FlashStateMachine.ScaleFclk.obj (.text:_scaleEEFclk)
                  0000e3e4    00000010                              : FlashStateMachine.ScaleFclk.obj (.text:_scaleMainFclk)
                  0000e3f4    0000000e     rtsv7R4_T_be_v3D16_eabi.lib : copy_decompress_none.obj (.text:decompress:none)
                  0000e402    0000000c     F021_API_CortexR4_BE.lib : Read.WdService.obj (.text:_Fapi_checkWdService)
                  0000e40e    0000000c     rtsv7R4_T_be_v3D16_eabi.lib : copy_zero_init.obj (.text:decompress:ZI)
                  0000e41a    00000002     --HOLE-- [fill = 0]
                  0000e41c    00000008     Fapi_UserDefinedFunctions.obj (.text)
                  0000e424    00000006     rtsv7R4_T_be_v3D16_eabi.lib : copy_decompress_rle.obj (.text:decompress:rle24)
                  0000e42a    00000002     --HOLE-- [fill = 0]
                  0000e42c    00000004     sys_phantom.obj (.text:retain)
                  0000e430    00000008     Fapi_UserDefinedFunctions.obj (.tramp.Fapi_serviceWatchdogTimer.1)

FEE_TEXT_SECTION 
*          0    0000e438    00002ec0     
                  0000e438    000011c0     ti_fee_writeSync.obj (FEE_TEXT_SECTION)
                  0000f5f8    00000cb8     ti_fee_writeAsync.obj (FEE_TEXT_SECTION)
                  000102b0    000007a8     ti_fee_read.obj (FEE_TEXT_SECTION)
                  00010a58    000004b0     ti_fee_format.obj (FEE_TEXT_SECTION)
                  00010f08    000003f0     ti_fee_invalidateblock.obj (FEE_TEXT_SECTION)

.const     0    000112f8    00000180     
                  000112f8    00000180     sys_vim.obj (.const:s_vim_init)

FEE_CONST_SECTION 
*          0    00011478    000000dc     
                  00011478    00000084     Device_TMS570LS31.obj (FEE_CONST_SECTION)
                  000114fc    00000058     ti_fee_cfg.obj (FEE_CONST_SECTION)

.cinit     0    00011558    00000050     
                  00011558    00000014     (.cinit..data.load) [load image, compression = rle]
                  0001156c    0000000c     (__TI_handler_table)
                  00011578    0000000b     (.cinit.FEE_DATA_SECTION.load) [load image, compression = rle]
                  00011583    00000005     --HOLE-- [fill = 0]
                  00011588    00000008     (.cinit..bss.load) [load image, compression = zero_init]
                  00011590    00000018     (__TI_cinit_table)

FEE_DATA_SECTION 
*          0    08001500    00000131     UNINITIALIZED
                  08001500    000000ff     ti_fee_ini.obj (FEE_DATA_SECTION)
                  080015ff    00000001     ti_fee_main.obj (FEE_DATA_SECTION)
                  08001600    00000028     ti_fee_util.obj (FEE_DATA_SECTION:uninit)
                  08001628    00000009     ti_fee_util.obj (FEE_DATA_SECTION:init)

.data      0    08001634    0000007e     UNINITIALIZED
                  08001634    00000064     sys_main.obj (.data:read_data)
                  08001698    00000008     F021_API_CortexR4_BE.lib : FlashStateMachine.ScaleFclk.obj (.data)
                  080016a0    00000008     rtsv7R4_T_be_v3D16_eabi.lib : _lock.obj (.data)
                  080016a8    00000008                                 : exit.obj (.data)
                  080016b0    00000001     F021_API_CortexR4_BE.lib : FlashStateMachine.SetActiveBank.obj (.data)
                  080016b1    00000001     sys_main.obj (.data)

.bss       0    080016b2    00000066     UNINITIALIZED
                  080016b2    00000064     sys_main.obj (.bss:SpecialRamBlock)
                  08001716    00000002     (.common:Status)

.TI.persistent 
*          0    08001634    00000000     UNINITIALIZED

.TI.noinit 
*          0    080016b2    00000000     UNINITIALIZED


LINKER GENERATED COPY TABLES

__TI_cinit_table @ 00011590 records: 3, size/record: 8, table size: 24
	.data: load addr=00011558, load size=00000014 bytes, run addr=08001634, run size=0000007e bytes, compression=rle
	FEE_DATA_SECTION: load addr=00011578, load size=0000000b bytes, run addr=08001500, run size=00000131 bytes, compression=rle
	.bss: load addr=00011588, load size=00000008 bytes, run addr=080016b2, run size=00000066 bytes, compression=zero_init


LINKER GENERATED HANDLER TABLE

__TI_handler_table @ 0001156c records: 3, size/record: 4, table size: 12
	index: 0, handler: __TI_zero_init
	index: 1, handler: __TI_decompress_rle24
	index: 2, handler: __TI_decompress_none

VENEERS

callee name               veneer name
   callee addr  veneer addr  call addr  call info
--------------  -----------  ---------  ----------------
Fapi_serviceWatchdogTimer  $Ven$TA$L$PI$$Fapi_serviceWatchdogTimer
   0000e41c     0000e430     0000e408   F021_API_CortexR4_BE.lib : Read.WdService.obj (.text:_Fapi_checkWdService)

[1 trampolines]
[1 trampoline calls]


GLOBAL SYMBOLS: SORTED ALPHABETICALLY BY Name 

address   name                                    
-------   ----                                    
0000e209  C$$EXIT                                 
00011478  Device_FlashDevice                      
0000e285  Fapi_calculateFletcherChecksum          
0000ddf9  Fapi_doBlankCheck                       
0000de8d  Fapi_enableEepromBankSectors            
0000e373  Fapi_flushPipeline                      
0000e3c5  Fapi_getNumberOfBankSectors             
0000d551  Fapi_initializeFlashBanks               
0000e129  Fapi_isAddressEcc                       
0000e349  Fapi_issueAsyncCommand                  
0000e2bd  Fapi_issueAsyncCommandWithAddress       
0000e41c  Fapi_serviceWatchdogTimer               
0000d7b1  Fapi_setActiveFlashBank                 
0000e2ed  Fapi_waitDelay                          
00011514  Fee_BlockConfiguration                  
000114fc  Fee_VirtualSectorConfiguration          
UNDEFED   SHT$$INIT_ARRAY$$Base                   
UNDEFED   SHT$$INIT_ARRAY$$Limit                  
080016b2  SpecialRamBlock                         
08001716  Status                                  
00000aec  TI_FeeInternal_AlignAddressForECC       
00001180  TI_FeeInternal_BlankCheck               
00005044  TI_FeeInternal_CheckForError            
00002b64  TI_FeeInternal_CheckModuleState         
00002bc4  TI_FeeInternal_CheckReadParameters      
000056e8  TI_FeeInternal_EnableRequiredFlashSector
00003158  TI_FeeInternal_FeeManager               
00000ebc  TI_FeeInternal_FindNextVirtualSector    
000051c4  TI_FeeInternal_Fletcher16               
00001d1c  TI_FeeInternal_GetArrayIndex            
00001c60  TI_FeeInternal_GetBlockIndex            
00001c24  TI_FeeInternal_GetBlockNumber           
00000e7c  TI_FeeInternal_GetBlockSize             
00002cf0  TI_FeeInternal_GetCurrentBlockAddress   
00001ce0  TI_FeeInternal_GetDataSetIndex          
00002df4  TI_FeeInternal_GetNextFlashAddress      
00001a48  TI_FeeInternal_GetVirtualSectorIndex    
00000020  TI_FeeInternal_GetVirtualSectorParameter
00004c1c  TI_FeeInternal_InvalidateErase          
00000e00  TI_FeeInternal_PollFlashStatus          
00002e40  TI_FeeInternal_SanityCheck              
00003030  TI_FeeInternal_SetClearCopyBlockState   
00004ed8  TI_FeeInternal_StartProgramBlock        
00001e8c  TI_FeeInternal_UpdateBlockOffsetArray   
000045c4  TI_FeeInternal_WriteBlockHeader         
00000664  TI_FeeInternal_WriteDataF021            
00000b24  TI_FeeInternal_WriteInitialize          
00004924  TI_FeeInternal_WritePreviousBlockHeader 
000001b8  TI_FeeInternal_WriteVirtualSectorHeader 
000052f0  TI_Fee_ErrorRecovery                    
080015fe  TI_Fee_FapiInitCalled                   
00010a58  TI_Fee_Format                           
00004fd8  TI_Fee_GetStatus                        
08001500  TI_Fee_GlobalVariables                  
0000856c  TI_Fee_Init                             
00010f08  TI_Fee_InvalidateBlock                  
00009c3c  TI_Fee_MainFunction                     
000102b0  TI_Fee_Read                             
000055b8  TI_Fee_SuspendResumeErase               
0000f5f8  TI_Fee_WriteAsync                       
0000e440  TI_Fee_WriteSync                        
080015e9  TI_Fee_bEraseSuspended                  
080015ea  TI_Fee_oStatusWord                      
080015e4  TI_Fee_u32ActCpyVS                      
080015dc  TI_Fee_u32BlockEraseCount               
080015d8  TI_Fee_u32FletcherChecksum              
080015d4  TI_Fee_u8DataSets                       
080015e0  TI_Fee_u8DeviceIndex                    
080015e8  TI_Fee_u8ErrEraseVS                     
080015ee  TI_FlashStatusWord                      
0000e1c5  _Fapi_EnableSectors                     
0000e403  _Fapi_checkWdService                    
0000e249  _Fapi_issueFsmCommand                   
0000e0cb  _Fapi_loopRegionForValue                
0000e31d  _Fapi_readDword                         
00011590  __TI_CINIT_Base                         
000115a8  __TI_CINIT_Limit                        
0001156c  __TI_Handler_Table_Base                 
00011578  __TI_Handler_Table_Limit                
0000d01c  __TI_PINIT_Base                         
0000d020  __TI_PINIT_Limit                        
0000dff5  __TI_auto_init                          
080016a8  __TI_cleanup_ptr                        
0000e3f5  __TI_decompress_none                    
0000e425  __TI_decompress_rle24                   
080016ac  __TI_dtors_ptr                          
00000000  __TI_static_base__                      
0000e40f  __TI_zero_init                          
0000df0d  __aeabi_memclr                          
0000df0d  __aeabi_memclr4                         
0000df0d  __aeabi_memclr8                         
0000dd5d  __aeabi_memcpy                          
0000dd5d  __aeabi_memcpy4                         
0000dd5d  __aeabi_memcpy8                         
0000df0f  __aeabi_memset                          
0000df0f  __aeabi_memset4                         
0000df0f  __aeabi_memset8                         
ffffffff  __binit__                               
ffffffff  __c_args__                              
0000d024  _c_int00                                
0000cf34  _coreClearAuxiliaryDataFault_           
0000cf48  _coreClearAuxiliaryInstructionFault_    
0000cf0c  _coreClearDataFaultAddress_             
0000cee4  _coreClearDataFault_                    
0000cf20  _coreClearInstructionFaultAddress_      
0000cef8  _coreClearInstructionFault_             
0000ce78  _coreDisableEventBusExport_             
0000cebc  _coreDisableFlashEcc_                   
0000ce98  _coreDisableRamEcc_                     
0000ce68  _coreEnableEventBusExport_              
0000cea8  _coreEnableFlashEcc_                    
0000cecc  _coreEnableIrqVicOffset_                
0000ce88  _coreEnableRamEcc_                      
0000ce50  _coreEnableVfp_                         
0000cf2c  _coreGetAuxiliaryDataFault_             
0000cf40  _coreGetAuxiliaryInstructionFault_      
0000cf04  _coreGetDataFaultAddress_               
0000cedc  _coreGetDataFault_                      
0000cf18  _coreGetInstructionFaultAddress_        
0000cef0  _coreGetInstructionFault_               
0000ccd8  _coreInitRegisters_                     
0000cde4  _coreInitStackPointer_                  
0000db94  _dabort                                 
0000cf5c  _disable_FIQ_interrupt_                 
0000cf64  _disable_IRQ_interrupt_                 
0000cf54  _disable_interrupt_                     
0000cf6c  _enable_interrupt_                      
0000cffc  _errata_CORTEXR4_57_                    
0000d00c  _errata_CORTEXR4_66_                    
0000cf74  _esmCcmErrorsClear_                     
0000ce30  _getCPSRValue_                          
0000ce38  _gotoCPUIdle_                           
080016a0  _lock                                   
0000e3bf  _nop                                    
0000dcd8  _pmuDisableCountersGlobal_              
0000dcc8  _pmuEnableCountersGlobal_               
0000dd34  _pmuGetCycleCount_                      
0000dd3c  _pmuGetEventCount_                      
0000dd48  _pmuGetOverflow_                        
0000dc7c  _pmuInit_                               
0000dd08  _pmuResetCounters_                      
0000dce8  _pmuResetCycleCounter_                  
0000dcf8  _pmuResetEventCounters_                 
0000dd28  _pmuSetCountEvent_                      
0000dd18  _pmuStartCounters_                      
0000dd20  _pmuStopCounters_                       
0000e3b7  _register_lock                          
0000e3b1  _register_unlock                        
0000e3d5  _scaleEEFclk                            
0000e3e5  _scaleMainFclk                          
080016a4  _unlock                                 
0000e20d  abort                                   
00006a5c  adc1ParityCheck                         
00006b48  adc2ParityCheck                         
ffffffff  binit                                   
00006c00  can1ParityCheck                         
00006cd8  can2ParityCheck                         
00006da0  can3ParityCheck                         
00005820  ccmSelfCheck                            
00007eec  ccmr4GetConfigValue                     
00006128  checkB0RAMECC                           
00006318  checkB1RAMECC                           
00007408  checkClockMonitor                       
00006508  checkFlashECC                           
000074e4  checkFlashEEPROMECC                     
0000767c  checkPLL1Slip                           
0000777c  checkPLL2Slip                           
00007840  checkRAMAddrParity                      
000071c0  checkRAMECC                             
0000794c  checkRAMUERRTest                        
00005fac  checkefcSelfTest                        
0000e179  copy_in                                 
00005a24  cpuSelfTest                             
000065ec  cpuSelfTestFail                         
000065e4  custom_dabort                           
00008348  disableParity                           
0000dfe0  dmaGroupANotification                   
0000669c  dmaParityCheck                          
00005e50  efcCheck                                
00007e50  efcGetConfigValue                       
00005f84  efcSelfTest                             
00005ed8  efcStuckZeroTest                        
000082c0  enableParity                            
00007f5c  errata_PBIST_4                          
0000c87c  esmActivateNormalOperation              
0000c960  esmClearStatus                          
0000c9ac  esmClearStatusBuffer                    
0000c840  esmDisableError                         
0000c8b8  esmDisableInterrupt                     
0000c814  esmEnableError                          
0000c88c  esmEnableInterrupt                      
0000caac  esmEnterSelfTest                        
0000c7f8  esmError                                
0000cb84  esmGetConfigValue                       
0000c9e8  esmGetStatus                            
0000ca74  esmGetStatusBuffer                      
0000df88  esmGroup1Notification                   
0000df98  esmGroup2Notification                   
0000da80  esmHighInterrupt                        
0000c6f0  esmInit                                 
0000cb34  esmSelfTestStatus                       
0000c9c8  esmSetCounterPreloadValue               
0000c8e4  esmSetInterruptLevel                    
0000c86c  esmTriggerErrorPinReset                 
0000e215  exit                                    
00007ab4  fmcBus1ParityCheck                      
0000604c  fmcBus2Check                            
00006088  fmcECCcheck                             
00006748  het1ParityCheck                         
000068b0  het2ParityCheck                         
000067f4  htu1ParityCheck                         
000069ac  htu2ParityCheck                         
0000d92c  main                                    
0000ae3c  mapClocks                               
0000dd5d  memcpy                                  
00005964  memoryInit                              
0000dfa8  memoryPort0TestFailNotification         
0000dfc4  memoryPort1TestFailNotification         
0000df15  memset                                  
00006e74  mibspi1ParityCheck                      
00006f7c  mibspi3ParityCheck                      
000070a0  mibspi5ParityCheck                      
0000c0c0  muxInit                                 
080016b1  oResult                                 
00007bdc  pbistFail                               
00007c60  pbistGetConfigValue                     
00005d98  pbistIsTestCompleted                    
00005dc4  pbistIsTestPassed                       
00005df8  pbistPortTestStatus                     
00005c9c  pbistRun                                
00005abc  pbistSelfCheck                          
00005d68  pbistStop                               
0000ade8  periphInit                              
0000e42c  phantomInterrupt                        
0000c444  pinmuxGetConfigValue                    
08001634  read_data                               
00000000  resetEntry                              
00005810  selftestFailNotification                
0000ada8  setupFlash                              
0000ad00  setupPLL                                
0000b620  sramGetConfigValue                      
00007dac  stcGetConfigValue                       
000059a8  stcSelfCheck                            
000065e8  stcSelfCheckFail                        
0000b060  systemGetConfigValue                    
0000af64  systemInit                              
0000b030  systemPowerDown                         
0000b474  tcmflashGetConfigValue                  
0000ad60  trimLPO                                 
0000b8fc  vimChannelMap                           
0000baf8  vimDisableInterrupt                     
0000b9a0  vimEnableInterrupt                      
0000bb7c  vimGetConfigValue                       
0000b828  vimInit                                 
000065f0  vimParityCheck                          
0000d2bc  vimParityErrorHandler                   


GLOBAL SYMBOLS: SORTED BY Symbol Address 

address   name                                    
-------   ----                                    
00000000  __TI_static_base__                      
00000000  resetEntry                              
00000020  TI_FeeInternal_GetVirtualSectorParameter
000001b8  TI_FeeInternal_WriteVirtualSectorHeader 
00000664  TI_FeeInternal_WriteDataF021            
00000aec  TI_FeeInternal_AlignAddressForECC       
00000b24  TI_FeeInternal_WriteInitialize          
00000e00  TI_FeeInternal_PollFlashStatus          
00000e7c  TI_FeeInternal_GetBlockSize             
00000ebc  TI_FeeInternal_FindNextVirtualSector    
00001180  TI_FeeInternal_BlankCheck               
00001a48  TI_FeeInternal_GetVirtualSectorIndex    
00001c24  TI_FeeInternal_GetBlockNumber           
00001c60  TI_FeeInternal_GetBlockIndex            
00001ce0  TI_FeeInternal_GetDataSetIndex          
00001d1c  TI_FeeInternal_GetArrayIndex            
00001e8c  TI_FeeInternal_UpdateBlockOffsetArray   
00002b64  TI_FeeInternal_CheckModuleState         
00002bc4  TI_FeeInternal_CheckReadParameters      
00002cf0  TI_FeeInternal_GetCurrentBlockAddress   
00002df4  TI_FeeInternal_GetNextFlashAddress      
00002e40  TI_FeeInternal_SanityCheck              
00003030  TI_FeeInternal_SetClearCopyBlockState   
00003158  TI_FeeInternal_FeeManager               
000045c4  TI_FeeInternal_WriteBlockHeader         
00004924  TI_FeeInternal_WritePreviousBlockHeader 
00004c1c  TI_FeeInternal_InvalidateErase          
00004ed8  TI_FeeInternal_StartProgramBlock        
00004fd8  TI_Fee_GetStatus                        
00005044  TI_FeeInternal_CheckForError            
000051c4  TI_FeeInternal_Fletcher16               
000052f0  TI_Fee_ErrorRecovery                    
000055b8  TI_Fee_SuspendResumeErase               
000056e8  TI_FeeInternal_EnableRequiredFlashSector
00005810  selftestFailNotification                
00005820  ccmSelfCheck                            
00005964  memoryInit                              
000059a8  stcSelfCheck                            
00005a24  cpuSelfTest                             
00005abc  pbistSelfCheck                          
00005c9c  pbistRun                                
00005d68  pbistStop                               
00005d98  pbistIsTestCompleted                    
00005dc4  pbistIsTestPassed                       
00005df8  pbistPortTestStatus                     
00005e50  efcCheck                                
00005ed8  efcStuckZeroTest                        
00005f84  efcSelfTest                             
00005fac  checkefcSelfTest                        
0000604c  fmcBus2Check                            
00006088  fmcECCcheck                             
00006128  checkB0RAMECC                           
00006318  checkB1RAMECC                           
00006508  checkFlashECC                           
000065e4  custom_dabort                           
000065e8  stcSelfCheckFail                        
000065ec  cpuSelfTestFail                         
000065f0  vimParityCheck                          
0000669c  dmaParityCheck                          
00006748  het1ParityCheck                         
000067f4  htu1ParityCheck                         
000068b0  het2ParityCheck                         
000069ac  htu2ParityCheck                         
00006a5c  adc1ParityCheck                         
00006b48  adc2ParityCheck                         
00006c00  can1ParityCheck                         
00006cd8  can2ParityCheck                         
00006da0  can3ParityCheck                         
00006e74  mibspi1ParityCheck                      
00006f7c  mibspi3ParityCheck                      
000070a0  mibspi5ParityCheck                      
000071c0  checkRAMECC                             
00007408  checkClockMonitor                       
000074e4  checkFlashEEPROMECC                     
0000767c  checkPLL1Slip                           
0000777c  checkPLL2Slip                           
00007840  checkRAMAddrParity                      
0000794c  checkRAMUERRTest                        
00007ab4  fmcBus1ParityCheck                      
00007bdc  pbistFail                               
00007c60  pbistGetConfigValue                     
00007dac  stcGetConfigValue                       
00007e50  efcGetConfigValue                       
00007eec  ccmr4GetConfigValue                     
00007f5c  errata_PBIST_4                          
000082c0  enableParity                            
00008348  disableParity                           
0000856c  TI_Fee_Init                             
00009c3c  TI_Fee_MainFunction                     
0000ad00  setupPLL                                
0000ad60  trimLPO                                 
0000ada8  setupFlash                              
0000ade8  periphInit                              
0000ae3c  mapClocks                               
0000af64  systemInit                              
0000b030  systemPowerDown                         
0000b060  systemGetConfigValue                    
0000b474  tcmflashGetConfigValue                  
0000b620  sramGetConfigValue                      
0000b828  vimInit                                 
0000b8fc  vimChannelMap                           
0000b9a0  vimEnableInterrupt                      
0000baf8  vimDisableInterrupt                     
0000bb7c  vimGetConfigValue                       
0000c0c0  muxInit                                 
0000c444  pinmuxGetConfigValue                    
0000c6f0  esmInit                                 
0000c7f8  esmError                                
0000c814  esmEnableError                          
0000c840  esmDisableError                         
0000c86c  esmTriggerErrorPinReset                 
0000c87c  esmActivateNormalOperation              
0000c88c  esmEnableInterrupt                      
0000c8b8  esmDisableInterrupt                     
0000c8e4  esmSetInterruptLevel                    
0000c960  esmClearStatus                          
0000c9ac  esmClearStatusBuffer                    
0000c9c8  esmSetCounterPreloadValue               
0000c9e8  esmGetStatus                            
0000ca74  esmGetStatusBuffer                      
0000caac  esmEnterSelfTest                        
0000cb34  esmSelfTestStatus                       
0000cb84  esmGetConfigValue                       
0000ccd8  _coreInitRegisters_                     
0000cde4  _coreInitStackPointer_                  
0000ce30  _getCPSRValue_                          
0000ce38  _gotoCPUIdle_                           
0000ce50  _coreEnableVfp_                         
0000ce68  _coreEnableEventBusExport_              
0000ce78  _coreDisableEventBusExport_             
0000ce88  _coreEnableRamEcc_                      
0000ce98  _coreDisableRamEcc_                     
0000cea8  _coreEnableFlashEcc_                    
0000cebc  _coreDisableFlashEcc_                   
0000cecc  _coreEnableIrqVicOffset_                
0000cedc  _coreGetDataFault_                      
0000cee4  _coreClearDataFault_                    
0000cef0  _coreGetInstructionFault_               
0000cef8  _coreClearInstructionFault_             
0000cf04  _coreGetDataFaultAddress_               
0000cf0c  _coreClearDataFaultAddress_             
0000cf18  _coreGetInstructionFaultAddress_        
0000cf20  _coreClearInstructionFaultAddress_      
0000cf2c  _coreGetAuxiliaryDataFault_             
0000cf34  _coreClearAuxiliaryDataFault_           
0000cf40  _coreGetAuxiliaryInstructionFault_      
0000cf48  _coreClearAuxiliaryInstructionFault_    
0000cf54  _disable_interrupt_                     
0000cf5c  _disable_FIQ_interrupt_                 
0000cf64  _disable_IRQ_interrupt_                 
0000cf6c  _enable_interrupt_                      
0000cf74  _esmCcmErrorsClear_                     
0000cffc  _errata_CORTEXR4_57_                    
0000d00c  _errata_CORTEXR4_66_                    
0000d01c  __TI_PINIT_Base                         
0000d020  __TI_PINIT_Limit                        
0000d024  _c_int00                                
0000d2bc  vimParityErrorHandler                   
0000d551  Fapi_initializeFlashBanks               
0000d7b1  Fapi_setActiveFlashBank                 
0000d92c  main                                    
0000da80  esmHighInterrupt                        
0000db94  _dabort                                 
0000dc7c  _pmuInit_                               
0000dcc8  _pmuEnableCountersGlobal_               
0000dcd8  _pmuDisableCountersGlobal_              
0000dce8  _pmuResetCycleCounter_                  
0000dcf8  _pmuResetEventCounters_                 
0000dd08  _pmuResetCounters_                      
0000dd18  _pmuStartCounters_                      
0000dd20  _pmuStopCounters_                       
0000dd28  _pmuSetCountEvent_                      
0000dd34  _pmuGetCycleCount_                      
0000dd3c  _pmuGetEventCount_                      
0000dd48  _pmuGetOverflow_                        
0000dd5d  __aeabi_memcpy                          
0000dd5d  __aeabi_memcpy4                         
0000dd5d  __aeabi_memcpy8                         
0000dd5d  memcpy                                  
0000ddf9  Fapi_doBlankCheck                       
0000de8d  Fapi_enableEepromBankSectors            
0000df0d  __aeabi_memclr                          
0000df0d  __aeabi_memclr4                         
0000df0d  __aeabi_memclr8                         
0000df0f  __aeabi_memset                          
0000df0f  __aeabi_memset4                         
0000df0f  __aeabi_memset8                         
0000df15  memset                                  
0000df88  esmGroup1Notification                   
0000df98  esmGroup2Notification                   
0000dfa8  memoryPort0TestFailNotification         
0000dfc4  memoryPort1TestFailNotification         
0000dfe0  dmaGroupANotification                   
0000dff5  __TI_auto_init                          
0000e0cb  _Fapi_loopRegionForValue                
0000e129  Fapi_isAddressEcc                       
0000e179  copy_in                                 
0000e1c5  _Fapi_EnableSectors                     
0000e209  C$$EXIT                                 
0000e20d  abort                                   
0000e215  exit                                    
0000e249  _Fapi_issueFsmCommand                   
0000e285  Fapi_calculateFletcherChecksum          
0000e2bd  Fapi_issueAsyncCommandWithAddress       
0000e2ed  Fapi_waitDelay                          
0000e31d  _Fapi_readDword                         
0000e349  Fapi_issueAsyncCommand                  
0000e373  Fapi_flushPipeline                      
0000e3b1  _register_unlock                        
0000e3b7  _register_lock                          
0000e3bf  _nop                                    
0000e3c5  Fapi_getNumberOfBankSectors             
0000e3d5  _scaleEEFclk                            
0000e3e5  _scaleMainFclk                          
0000e3f5  __TI_decompress_none                    
0000e403  _Fapi_checkWdService                    
0000e40f  __TI_zero_init                          
0000e41c  Fapi_serviceWatchdogTimer               
0000e425  __TI_decompress_rle24                   
0000e42c  phantomInterrupt                        
0000e440  TI_Fee_WriteSync                        
0000f5f8  TI_Fee_WriteAsync                       
000102b0  TI_Fee_Read                             
00010a58  TI_Fee_Format                           
00010f08  TI_Fee_InvalidateBlock                  
00011478  Device_FlashDevice                      
000114fc  Fee_VirtualSectorConfiguration          
00011514  Fee_BlockConfiguration                  
0001156c  __TI_Handler_Table_Base                 
00011578  __TI_Handler_Table_Limit                
00011590  __TI_CINIT_Base                         
000115a8  __TI_CINIT_Limit                        
08001500  TI_Fee_GlobalVariables                  
080015d4  TI_Fee_u8DataSets                       
080015d8  TI_Fee_u32FletcherChecksum              
080015dc  TI_Fee_u32BlockEraseCount               
080015e0  TI_Fee_u8DeviceIndex                    
080015e4  TI_Fee_u32ActCpyVS                      
080015e8  TI_Fee_u8ErrEraseVS                     
080015e9  TI_Fee_bEraseSuspended                  
080015ea  TI_Fee_oStatusWord                      
080015ee  TI_FlashStatusWord                      
080015fe  TI_Fee_FapiInitCalled                   
08001634  read_data                               
080016a0  _lock                                   
080016a4  _unlock                                 
080016a8  __TI_cleanup_ptr                        
080016ac  __TI_dtors_ptr                          
080016b1  oResult                                 
080016b2  SpecialRamBlock                         
08001716  Status                                  
ffffffff  __binit__                               
ffffffff  __c_args__                              
ffffffff  binit                                   
UNDEFED   SHT$$INIT_ARRAY$$Base                   
UNDEFED   SHT$$INIT_ARRAY$$Limit                  

[256 symbols]
